:100000000C94E6030C940E040C940E040C940E0451
:100010000C940E040C940E040C940E040C940E0418
:100020000C940E040C940E040C940E040C940E0408
:100030000C940E040C940E040C940E040C940E04F8
:100040000C946D0C0C940E040C940E040C940E0481
:100050000C940E040C940E040C940E040C940E04D8
:100060000C940E040C940E0400000000003E5B4F44
:100070005B3E3E6B4F6B3E1C3E7C3E1C183C7E3C08
:10008000181C577D571C1C5E7F5E1C00183C180016
:10009000FFE7C3E7FF0018241800FFE7DBE7FF30A6
:1000A000483A060E2629792926407F050507407F14
:1000B00005253F5A3CE73C5A7F3E1C1C08081C1C87
:1000C0003E7F14227F22145F5F005F5F06097F017D
:1000D0007F006689956A606060606094A2FFA29468
:1000E00008047E040810207E201008082A1C080836
:1000F0001C2A08081E101010100C1E0C1E0C303884
:100100003E3830060E3E0E06000000000000005F84
:1001100000000007000700147F147F14242A7F2AA0
:100120001223130864623649562050000807030062
:10013000001C2241000041221C002A1C7F1C2A08AE
:10014000083E080800807030000808080808000011
:1001500060600020100804023E5149453E00427F85
:10016000400072494949462141494D331814127FD4
:100170001027454545393C4A494931412111090774
:100180003649494936464949291E000014000000F5
:1001900040340000000814224114141414140041C7
:1001A00022140802015909063E415D594E7C121184
:1001B000127C7F494949363E414141227F414141BC
:1001C0003E7F494949417F090909013E4141517337
:1001D0007F0808087F00417F41002040413F017FA8
:1001E000081422417F404040407F021C027F7F0470
:1001F00008107F3E4141413E7F090909063E4151B9
:10020000215E7F09192946264949493203017F01A8
:10021000033F4040403F1F2040201F3F4038403FA9
:10022000631408146303047804036159494D4300BF
:100230007F4141410204081020004141417F0402F6
:10024000010204404040404000030708002054548D
:1002500078407F284444383844444428384444286B
:100260007F385454541800087E090218A4A49C78BE
:100270007F0804047800447D40002040403D007F1A
:100280001028440000417F40007C047804787C08FA
:100290000404783844444438FC18242418182424CE
:1002A00018FC7C08040408485454542404043F44B3
:1002B000243C4040207C1C2040201C3C4030403CE2
:1002C00044281028444C9090907C4464544C440042
:1002D00008364100000077000000413608000201A6
:1002E0000204023C2623263C1EA1A161123A404092
:1002F000207A38545455592155557941225454780F
:1003000042215554784020545579400C1E527212A7
:100310003955555559395454545939555454580030
:1003200000457C410002457D420001457C407D1234
:1003300011127DF0282528F07C5455450020545496
:100340007C547C0A097F4932494949323A44444441
:100350003A324A4848303A4141217A3A424020787C
:10036000009DA0A07D3D4242423D3D4040403D3C7D
:1003700024FF2424487E4943662B2FFC2F2BFF09A2
:1003800029F620C0887E0903205454794100004496
:100390007D413048484A32384040227A007A0A0A81
:1003A000727D0D19317D2629292F282629292926F4
:1003B00030484D4020380808080808080808382F39
:1003C00010C8ACBA2F102834FA00007B00000814C3
:1003D0002A142222142A14085500550055AA55AA99
:1003E00055AAFF55FF55FF000000FF00101010FF39
:1003F00000141414FF001010FF00FF1010F010F094
:10040000141414FC001414F700FF0000FF00FF1484
:1004100014F404FC141417101F10101F101F1414D0
:10042000141F00101010F0000000001F101010101A
:100430001F10101010F010000000FF10101010100E
:1004400010101010FF10000000FF140000FF00FF4C
:1004500000001F10170000FC04F4141417101714E8
:1004600014F404F40000FF00F7141414141414140A
:10047000F700F7141414171410101F101F1414147D
:10048000F4141010F010F000001F101F0000001FE7
:1004900014000000FC140000F010F01010FF10FF1A
:1004A000141414FF141010101F00000000F010FFAF
:1004B000FFFFFFFFF0F0F0F0F0FFFFFF0000000093
:1004C00000FFFF0F0F0F0F0F3844443844FC4A4A17
:1004D0004A347E02020606027E027E0263554941CC
:1004E000633844443C04407E201E2006027E020203
:1004F00099A5E7A5991C2A492A1C4C7201724C3017
:100500004A4D4D303048784830BC625A463D3E49ED
:100510004949007E0101017E2A2A2A2A2A44445F91
:10052000444440514A444040444A51400000FF0185
:1005300003E080FF000008086B6B08361236243693
:10054000060F090F060000181800000010100030F8
:1005500040FF0101001F01011E00191D1712003C80
:100560003C3C3C00000000000000000800020100CC
:10057000000304070000000000000000000000006D
:10058000000000000000000000000000000000006B
:10059000000000000000000000000000000000005B
:1005A000000000000000000000000000000000004B
:1005B00000000000000000007000000000000000CB
:1005C000000001FC00000000000000000007FF0028
:1005D00000000000000000003FFFC000000000001D
:1005E000000000FFFFF00000000000000003F16CBD
:1005F000FE000000000000000FC0F83F8000000077
:100600000000003300700FE0000000000000F80060
:100610006000F8000000000003FA007001FE000016
:100620000000000FC100FC043F80000000003F00FC
:1006300007FF0807E000000000FC002E07A001F8FB
:1006400000000003F0001803C0007E0000000FC08F
:100650000011FCC0001F8000003F00003100E000DE
:1006600007E00000F800002103F00001F80002F0AC
:1006700000002103F0000066001CFFFFFE20FFF7D2
:10068000FFFFF1800EE0000C1CBFF3000037800379
:100690000000080CFFF100000E0000C8001026FF4B
:1006A000B080003800003000200603A04000C000E9
:1006B000000C000006FF60000300000001000003C2
:1006C000FEC0000C00000000413F09FD8FC8300053
:1006D000000000110006070000C00000000005C077
:1006E00003FE001B000000000001E00060007C0031
:1006F0000000000000E0006000700000000000004A
:1007000018006001C00000000000000E40600700FB
:100710000000000000000390607C0000000000006A
:100720000000FEF1F000000000000000003FFFC0EC
:10073000000000000000000007FF000000000000B3
:1007400000000001FC00000000000000000000604C
:100750000000000000000000000000000000000099
:100760000000000000000000000000000000000089
:100770000000000000000000000000000000000079
:100780000000000000000000000000000000000069
:10079000250028002B0000000000240027002A006C
:1007A0000404040404040404020202020202030317
:1007B000030303030102040810204080010204081F
:1007C0001020010204081020EC0E2B0F11241FBE74
:1007D000CFEFD8E0DEBFCDBF23E0AAE3B3E001C096
:1007E0001D92AB37B207E1F713E0A0E0B1E0E8E714
:1007F000F3E202C005900D92AA33B107D9F713E0D6
:10080000C5EED3E004C02197FE010E949D0FC43EB7
:10081000D107C9F70E94B70C0C94AF110C940000DB
:10082000909168039F3F21F4909169039F3F59F194
:1008300028E030E040E8E0917303F09174035081C8
:1008400090917603909595239083E0917103F091B8
:10085000720390917503542F582319F05081952BF2
:1008600003C05081909595239083E0917303F0919C
:100870007403508190917603952B90834695215077
:100880003109C9F608958EBD00000DB407FEFDCFF5
:100890008EB5089590E0FC01EC54F84F2491FC01D2
:1008A000E056F84F8491882399F090E0880F991FC3
:1008B000FC01EA56F84FA591B491FC01E457F84FBA
:1008C000859194918FB7F894EC91E22BEC938FBFC4
:1008D0000895089508950895CF92DF92EF92FF92C0
:1008E0000F931F93CF93DF936C017A018B01C0E0CC
:1008F000D0E0CE15DF0589F0D8016D918D01D601CC
:10090000ED91FC910190F081E02DC6010995892BB4
:1009100011F47E0102C02196ECCFC701DF91CF9187
:100920001F910F91FF90EF90DF90CF90089590E08E
:10093000FC01E859FA4F3491FC01EC54F84F249132
:10094000FC01E056F84FE491EE2309F43BC0332359
:1009500039F1333091F038F43130A9F0323001F50B
:1009600084B58F7D12C0373091F03830A1F034302B
:10097000B9F4809180008F7D03C0809180008F77D3
:10098000809380000DC084B58F7784BD09C08091AD
:10099000B0008F7703C08091B0008F7D8093B0004E
:1009A000F0E0EE0FFF1FE457F84FA591B4918FB719
:1009B000F894EC91611103C020952E2301C02E2BD9
:1009C0002C938FBF0895CF93C82F60E080916A0366
:1009D0000E94970480916C0318161CF460E00E943A
:1009E00097048C2F0E94100480916C03181624F435
:1009F00061E0CF910C949704CF910895CF93C82FC5
:100A000087FDCFE7C0936D0381E20E94E3048C2F42
:100A100080680E94E30480E2CF910C94E3043FB726
:100A2000F89480913F0390914003A0914103B091CD
:100A3000420326B5A89B05C02F3F19F00196A11DC2
:100A4000B11D3FBFBA2FA92F982F8827820F911D64
:100A5000A11DB11DBC01CD0142E0660F771F881FAB
:100A6000991F4A95D1F708958F929F92AF92BF92A6
:100A7000CF92DF92EF92FF926B017C010E940F05F3
:100A80004B015C01C114D104E104F104F1F00E94B6
:100A90000F05DC01CB0188199909AA09BB09883E19
:100AA0009340A105B10570F321E0C21AD108E10815
:100AB000F10888EE880E83E0981EA11CB11CC114B9
:100AC000D104E104F10419F7DDCFFF90EF90DF903E
:100AD000CF90BF90AF909F908F900895CF938091CB
:100AE0006B03181674F460E00E94970464EF71E0E1
:100AF00080E090E00E94340561E080916B030E94E9
:100B00009704C0916E03C83008F0C7E0C0936E032D
:100B100081E20E94E3048C2F80610E94E30480E262
:100B20000E94E30480916D030E94FE0480E20E9413
:100B3000E3048CE0CF910C94E304EF92FF920F93C7
:100B40001F93CF9390916F03992361F0809170036D
:100B50008F5F891718F48093700304C0109270039C
:100B60000E946E0580E0E82E81E0F82EC0E08C2F18
:100B700080640E94E30480E80E94E30461E08091C5
:100B80006A030E94970480916C0318161CF460E0BD
:100B90000E94970400E010E0F701E00FF11F808150
:100BA0000E9410040F5F1F4F04351105A9F78091B3
:100BB0006C0318161CF461E00E949704CF5F84E573
:100BC000E80EF11CC63099F680E4CF911F910F9189
:100BD000FF90EF900C94E304FC0177FD68C08085E2
:100BE0009185681779070CF062C057FD60C0828557
:100BF0009385481759070CF05AC08689823059F0FE
:100C00008330B1F08130D1F48FE290E0861B970BF6
:100C1000BA01AC0113C083E590E0FC01E61BF70BC1
:100C2000BF018FE290E0FC01E41BF50BAF0106C0B1
:100C300083E590E0841B950BAB01BC016435710525
:100C4000B0F54033510598F5CA01E3E095958795D5
:100C5000EA95E1F747705527232BA1F024E5289F5B
:100C6000F001299FF00D11246E0F7F1FFB01E05052
:100C7000FF4F81E090E001C0880F4A95EAF790812C
:100C8000892B14C024E5289FF001299FF00D112421
:100C90006E0F7F1FFB01E050FF4F81E090E001C02D
:100CA000880F4A95EAF7809590818923808308957B
:100CB0000895FC016370668B84819581268137815C
:100CC000613039F0633029F091878087338722873C
:100CD0000895318720879387828708952F923F92C6
:100CE0004F925F926F927F928F929F92AF92BF923C
:100CF000CF92DF92EF92FF920F931F93CF93DF93E8
:100D0000CDB7DEB76C970FB6F894DEBF0FBECDBF80
:100D10009C8F8B8F1B014A01198708873701A98295
:100D2000DC0159964D915C915A974115510509F096
:100D3000FFC018968D919C911997681779070CF050
:100D4000E1C11A968D919C911B97881699060CF01B
:100D5000D9C1EC2DF0E0FB83EA83AB0166E0C69ECF
:100D6000400D511D11245D874C87141615060CF09B
:100D7000C9C18A2D90E09B878A8733E0880F991F2D
:100D80003A95E1F79F878E87880D991D18161906E9
:100D90000CF0B8C158968C91811103C0203B08F02B
:100DA0002F5FAB8DBC8DED91FC9111970680F78183
:100DB000E02DCD012A8F09952A8DB5E02B9F90015A
:100DC0001124EC2DF0E0F98BE88BA1014B5F5F4F14
:100DD0005B8B4A8B3D822C822101B9016219730918
:100DE0007D8B6C8B9981892F90E09F8B8E8BD401AA
:100DF0001896B98FA88FEC89FD89E40DF51DE85987
:100E0000FF4FD49054019F828E82D0FE16C0AB8DCE
:100E1000BC8DED91FC91B1E0CB1209C0298121304C
:100E200031F40084F185E02D2885398519C00284CC
:100E3000F385E02DE884F9841DC048855985641642
:100E4000750619F1AB8DBC8DED91FC91B1E0CB1223
:100E50000DC02981213051F40084F185E02D9301EA
:100E6000A501B2018B8D9C8D09950FC00284F3857D
:100E7000E02D73010A851B852A813B814E815F81AC
:100E80006C817D818B8D9C8D0995D6943FEFA31A43
:100E9000B30A4E815F816E897F89460F571F5F833A
:100EA0004E83888D998DA816B90609F0AECF9FEFB5
:100EB000491A590AAC81BD81E889F989AE0FBF1F73
:100EC000BD83AC832A893B894216530609F093CF30
:100ED000488559856416750609F4F2C0AB8DBC8D42
:100EE000ED91FC91B1E0CB1211C02981213071F458
:100EF000B1016B5F7F4F0484F585E02D830128E00D
:100F000030E0A4018B8D9C8D0995DAC06C857D85C0
:100F10004A815B81641B750B0284F385E02D7301AC
:100F20000E851F859A01A4018B8D9C8D0995C8C0E3
:100F3000FA0134969491329765917491291BCB01F3
:100F4000B7E02B9F800D911D1124FA01259134915A
:100F50003B8B2A8BFC01A590B490FC0132965490F7
:100F6000319634913C87329614913196749041E0D9
:100F70004C1518F05981523068F0612F012E000C89
:100F8000770B7B836A83872D072C000C990B9D833D
:100F90008C8304C01D821C821B821A82AB8DBC8D87
:100FA000ED91FC9111970680F781E02DCD01099517
:100FB000412CD12C612CF981EF2FF0E0FF83EE83DF
:100FC0002C2D30E03B872A87A401470D511D77FC6B
:100FD0005A955F8B4E8BB101610F711D17FD7A958C
:100FE000798F688F5C85651608F06AC0262D30E021
:100FF0004C815D81420F531F6E817F81469FC001EE
:10100000479F900D569F900D1124DC01A80DB91D2E
:10101000B98BA88B842D712CEE89FF89E20FF31F09
:10102000FD8BEC8B751408F048C071E0780F7E875B
:10103000877041F4C5010196EA89FB89EA0DFB1D21
:10104000D4905C01D7FE35C0AB8DBC8DED91FC9189
:10105000B1E0CB1212C02981213079F40084F185EE
:10106000E02D288539854C895D89688D798D670DDE
:10107000711D8B8D9C8D09951CC08A819B81870D6C
:10108000911D4A855B85849FB001859F700D949F5B
:10109000700D1124620D731D0284F385E02DE88428
:1010A000F9840E811F819A01488959898B8D9C8D05
:1010B0000995DD0C73948E85B5CF450C639492CF62
:1010C000AB8DBC8DED91FC9111970288F389E02DD9
:1010D000CD016C960FB6F894DEBF0FBECDBFDF9189
:1010E000CF911F910F91FF90EF90DF90CF90BF9025
:1010F000AF909F908F907F906F905F904F903F90B8
:101100002F9009946C960FB6F894DEBF0FBECDBF3A
:10111000DF91CF911F910F91FF90EF90DF90CF90D3
:10112000BF90AF909F908F907F906F905F904F9007
:101130003F902F9008958F929F92AF92CF92EF920F
:10114000FF920F931F93CF93DF93EC01262F898D8E
:101150009A8D009709F042C06A3059F41D861C86AA
:101160002D898E859F8538E0239F800D911D112448
:1011700043C06D3009F4AAC08F898823C9F03C8927
:101180008C859D8546E0349F800D911D11244885F6
:1011900059854817590764F41D861C863D898E853C
:1011A0009F8548E0349F800D911D11249F878E8775
:1011B000EA88FB88088919894E855F856C857D855D
:1011C000AD88CC88CE010E946E062C898C859D85C9
:1011D00036E0239F800D911D11243EC06A3079F4C2
:1011E0001D861C862D89FC013696E4918E859F858F
:1011F0002E9F800D911D11249F878E8767C06D30B3
:1012000009F464C0FC0134963491631708F45EC09D
:101210003196E491E61708F459C0462F431B342F4A
:10122000FC0132968590949047E0349F800C911C8D
:101230001124F401329634913196E491332311F064
:10124000E1110DC0F4013496E4912C898C859D85C3
:10125000E29F800D911D11249D878C8737C0F4017A
:10126000359644915F89552319F15C89E32FF0E0AD
:10127000E40FF11D47FDFA955E9FB0015F9F700D71
:1012800011244C855D85460F571F68857985641745
:10129000750774F41D861C863D89FC013696E49121
:1012A0008E859F853E9F800D911D11249F878E877F
:1012B000EA88FB88088919894E855F856C857D855C
:1012C000AD88CC88CE010E946E06BCCF81E090E054
:1012D000DF91CF911F910F91FF90EF90CF90AF9042
:1012E0009F908F9008956F927F928F929F92AF926E
:1012F000BF92CF92DF92EF92FF920F931F93CF9303
:10130000DF93EC014B015A0169013801E881F98151
:101310000680F781E02D0995E881F9810684F7853B
:10132000E02D87019601A501B401CE010995E88160
:10133000F981A501460D571D415051090684F785D5
:10134000E02D9601B401CE010995E881F98104846C
:10135000F585E02D9301A501B401CE010995E88141
:10136000F981C80CD91CB601615071090484F58556
:10137000E02D9301A501CE010995E881F98102884C
:10138000F389E02DCE01DF91CF911F910F91FF9056
:10139000EF90DF90CF90BF90AF909F908F907F9015
:1013A0006F900994CF92DF92EF92FF920F931F9369
:1013B000CF93DF9300D000D000D0CDB7DEB76C0163
:1013C000DC01ED91FC916217730789F4041715078E
:1013D0002CF4942F852FA801092F182F041B150B0F
:1013E00098012F5F3F4F008CF18DE02D12C0401708
:1013F000510709F5261737072CF4962F872FB901C7
:10140000292F382F261B370B2F5F3F4F028CF38D70
:10141000E02D8701C601099526960FB6F894DEBF28
:101420000FBECDBFDF91CF911F910F91FF90EF9035
:10143000DF90CF9008950680F781E02D2D833E83C5
:101440004B835C8369837A830995D601ED91FC9186
:101450000088F189E02D2D813E814B815C8169817D
:101460007A81C6010995D601ED91FC910288F38934
:10147000E02DC60126960FB6F894DEBF0FBECDBF95
:10148000DF91CF911F910F91FF90EF90DF90CF9060
:101490000994EF92FF920F931F93DC01ED91FC9161
:1014A00011971A960D911C911B9718962D913C91AE
:1014B0001997048CF58DE02D7B0140E050E060E051
:1014C00070E009951F910F91FF90EF9008954F9252
:1014D0005F926F927F928F929F92AF92BF92CF92C4
:1014E000DF92EF92FF920F931F93CF93DF9300D081
:1014F000CDB7DEB76C015A0139014801DC01ED912D
:10150000FC910680F781E02D69837A8309956981D2
:10151000462E7A81572E640C751CD601ED91FC91F4
:10152000461457046CF40484F585E02D870194017A
:10153000A501B201C6010995BFEF4B1A5B0AEDCFB9
:101540000288F389E02DC6010F900F90DF91CF91B3
:101550001F910F91FF90EF90DF90CF90BF90AF90D1
:101560009F908F907F906F905F904F900994AF9273
:10157000BF92CF92DF92EF92FF920F931F93CF9380
:10158000DF9300D000D0CDB7DEB75C016901DC018C
:10159000ED91FC910680F781E02D4B835C8369839C
:1015A0007A830995D501ED91FC9169817A819B013E
:1015B0002C0D3D1D215031090088F189E02D780165
:1015C0004B815C818A01C5010995D501ED91FC91A2
:1015D0000288F389E02DC5010F900F900F900F90B6
:1015E000DF91CF911F910F91FF90EF90DF90CF90FF
:1015F000BF90AF900994AF92BF92CF92DF92EF92DB
:10160000FF920F931F93CF93DF9300D000D0CDB7FD
:10161000DEB75C016901DC01ED91FC910680F78188
:10162000E02D4B835C8369837A830995D501ED9125
:10163000FC914B815C81C40ED51EB1E0CB1AD10860
:101640000088F189E02D7801860169817A819B010A
:10165000C5010995D501ED91FC910288F389E02D32
:10166000C5010F900F900F900F90DF91CF911F91B8
:101670000F91FF90EF90DF90CF90BF90AF900994C3
:10168000EF92FF920F931F93DC01ED91FC91048C7C
:10169000F58DE02D09951F910F91FF90EF90089522
:1016A0000F931F93DC01ED91FC91028CF38DE02DE3
:1016B00009951F910F9108950F931F93DC01ED91F0
:1016C000FC91008CF18DE02D09951F910F910895EB
:1016D000DC01ED91FC910480F581E02D09942F92BD
:1016E0003F924F925F926F927F928F929F92AF92B2
:1016F000BF92CF92DF92EF92FF920F931F93CF93FF
:10170000DF9300D01F92CDB7DEB74C017B836A8395
:101710006A01590117019801241B350B37FF03C0DB
:10172000319521953109C5014A815B81841B950B57
:1017300097FF03C091958195910951E059838217D4
:10174000930714F019820BC09A2D8B2D5801092F85
:10175000182F9A818B81DB82CA82C92ED82E8A816A
:101760009B81A816B9065CF49C2D8D2D6801092F6C
:10177000182F9A818B81BB82AA82A92EB82E2501AF
:10178000AA81BB814A1A5B0A38016C187D0877FE72
:1017900003C0719461947108720157FE03C0BFEFDA
:1017A000EB1AFB0AF594E794C016D1061CF00FEF74
:1017B0001FEF1FC001E010E01CC0D401ED91FC91AF
:1017C000B9810084F185E02D9101BB23C1F04A81EC
:1017D0005B81B601C4010995E618F708F7FE04C05D
:1017E000C00ED11EE40CF51CEA81FB813196FB830F
:1017F000EA834A815B81A416B506FCF604C0A60103
:101800006A817B81E7CF0F900F900F90DF91CF918E
:101810001F910F91FF90EF90DF90CF90BF90AF900E
:101820009F908F907F906F905F904F903F902F9000
:101830000895009769F0FC0101900020E9F73197C5
:10184000AF01481B590BBC018DE493E00C946C0470
:1018500080E090E008950E949A11EF92FF920F931A
:101860001F93CF93DF93EC017B018A0188819981DB
:10187000009729F02A813B8124173507F8F4B80135
:101880006F5F7F4F0E94D010009759F09983888333
:101890001B830A832C813D81232B81F4FC01108260
:1018A0000DC088819981009711F00E94381019822B
:1018B00018821D821C821B821A8207C01D830C8322
:1018C000B701888199810E94A811CE01DF91CF9143
:1018D0001F910F91FF90EF9008951F920F920FB6F6
:1018E0000F9211242F933F938F939F93AF93BF93A6
:1018F00080913B0390913C03A0913D03B0913E0346
:1019000030913A0323E0230F2D3720F40196A11DD7
:10191000B11D05C026E8230F0296A11DB11D20931D
:101920003A0380933B0390933C03A0933D03B09311
:101930003E0380913F0390914003A0914103B091F9
:1019400042030196A11DB11D80933F039093400374
:10195000A0934103B0934203BF91AF919F918F91A8
:101960003F912F910F900FBE0F901F901895CF931E
:10197000DF93CDB7DEB768970FB6F894DEBF0FBE22
:10198000CDBF789484B5826084BD84B5816084BD08
:1019900085B5826085BD85B5816085BD80916E000D
:1019A000816080936E00109281008091810082603E
:1019B000809381008091810081608093810080917B
:1019C00080008160809380008091B100846080936A
:1019D000B1008091B00081608093B00080917A0066
:1019E000846080937A0080917A00826080937A008C
:1019F00080917A00816080937A0080917A0080687B
:101A000080937A001092C100809168038F3F29F47F
:101A1000909169039F3F09F4A2C10E944A048091FA
:101A200069030E944A0480916903082E000C990BF7
:101A3000FC01E056F84FE491F0E0EE0FFF1FE45791
:101A4000F84F259134913093740320937303FC0174
:101A5000EC54F84FE491E093760380916803082EEC
:101A6000000C990BFC01E056F84FE491F0E0EE0F0A
:101A7000FF1FE457F84F2591349130937203209360
:101A80007103FC01EC54F84FE491E09375038091ED
:101A90006A030E944A0480916B03181614F40E9492
:101AA0004A0480916C03181614F40E944A0484E0DE
:101AB00080936E0388E280936D0310926F031092FF
:101AC00070030E946E050E949D0582E30E94FE0441
:101AD00088EF91E0E0E0F1E0DF019C011D922150F0
:101AE0003040E1F781E0809361038093620381E0FD
:101AF00090E09093600380935F0390935E038093E4
:101B00005D032AE030E030935A0320935903909309
:101B10005C0380935B0386E293E00E94190C82E3EE
:101B200093E00E94190C612C712CD12C05E010E07F
:101B3000812C912CC40187709927892B11F0DD0C21
:101B40000BC0F40173E0F595E7957A95E1F7E60DA2
:101B5000F71DE458FA4FD490D7FE08C021E030E0DA
:101B6000A801B4018DE493E00E94680B3FEF831A53
:101B7000930A48E584169104E9F60F5F1F4F5BE076
:101B8000650E711C0533110599F60E949D0560EDE7
:101B900077E080E090E00E94340510925A031092A2
:101BA00059038AE090E090935C0380935B0385E3A4
:101BB00093E00E94190C0E949D0560ED77E080E0A3
:101BC00090E00E943405CE0101963C0144244394E8
:101BD000512C56E0D52E60E0262E60E0362E809106
:101BE0004B0390914C03019690934C0380934B03CD
:101BF0001C8A1B8A1E8A1D8A188E1F8A4AE0B3011E
:101C00000E94310FF30101900020E9F73197AF01F5
:101C100046195709B301CE0143960E942D0C8091BD
:101C20004503909146030097C9F06B897C89611543
:101C3000710591F040914703509148032F89388DE9
:101C40004217530748F00E94A8118F89988D9093EE
:101C50004A038093490318C00E9438108B899C89DD
:101C600090934603809345038D899E899093480302
:101C7000809347038F89988D90934A0380934903FB
:101C80001C8A1B8A1E8A1D8A188E1F8A8B899C8932
:101C90000E943810812C912CAA24A394CC24C394A4
:101CA000E12CF12C0FEF10E020E24AE050E0B4010B
:101CB0008DE493E00E946E0696E0890E911CA8E1E7
:101CC0008A16910449F78090490390904A03B1E045
:101CD0008B1A910897FC34C08091490390914A0374
:101CE0008816990630F4E0914503F0914603309749
:101CF00029F410924403E4E4F3E002C0E80DF91D76
:101D00002081A201481B590BCA01880D991DD89E3C
:101D1000B001D99E700D11246E5E7F4FAA24A3944A
:101D2000CC24C394E12CF12C0FEF10E04AE050E0FA
:101D30008DE493E00E946E0651E0851A9108CACFA7
:101D40000E949D0564EF71E080E090E00E94340500
:101D50002114310409F443CF0E94000040CF1FB783
:101D6000F89480914303811124C0EAEAF7E084915A
:101D7000EEEBF7E09491E82FF0E0EE0FFF1FEA564C
:101D8000F84FA591B491EC91E92321F461E08AE048
:101D90000E9497048AE00E944A048CB580618CBD41
:101DA0008CB580648CBD8DE00E944A048BE00E945B
:101DB0004A04809143038F5F809343031FBF8CB518
:101DC0008C7F8CBD8DB58E7F8DBD8CB5837F8CBD9A
:101DD0008CB58F7D8CBD5BCEEDE4F3E01382128277
:101DE00024E530E03583248380E390E09783868385
:101DF0003187208793878287168A158614861786EF
:101E0000168681E0858B848B2FEF3FEF338B228BFF
:101E1000318B208B878B108E128E118E82E093E097
:101E20009183808380E1838F81E1848F8FE0858F30
:101E30008EE0868F8FEF878FE5E4F3E011821082CA
:101E4000138212821582148240E050E064E373E052
:101E5000CF010C942D0C80914503909146030C9476
:101E60003810BB274A3031F4992322F4BDE2909513
:101E700081959F4F0C943D0FBB27FB015527AA2747
:101E8000880F991FAA1FA41710F0A41B8395505107
:101E9000B9F7A05DAA3308F0A95DA193009779F77F
:101EA000B111B1931192CB010C94560FDC01FC01DE
:101EB000672F71917723E1F7329704C07C916D937E
:101EC00070836291AE17BF07C8F308952F923F92B7
:101ED0004F925F926F927F928F929F92AF92BF923A
:101EE000CF92DF92EF92FF920F931F93CF93DF93E6
:101EF000CDB7DEB7CA1BDB0B0FB6F894DEBF0FBE43
:101F0000CDBF09942A88398848885F846E847D848F
:101F10008C849B84AA84B984C884DF80EE80FD8091
:101F20000C811B81AA81B981CE0FD11D0FB6F89407
:101F3000DEBF0FBECDBFED010895EE0FFF1F059070
:101F4000F491E02D0994CF93DF938230910510F442
:101F500082E090E0E0917903F0917A0320E030E0B4
:101F6000C0E0D0E0309711F1408151814817590706
:101F7000C0F04817590761F482819381209719F0C6
:101F80009B838A832BC090937A038093790326C026
:101F90002115310519F04217530718F49A01BE01B3
:101FA000DF01EF010280F381E02DDCCF2115310547
:101FB00009F1281B390B2430310590F412968D91CC
:101FC0009C9113976115710521F0FB019383828326
:101FD00004C090937A0380937903FD01329644C044
:101FE000FD01E20FF31F81939193225031092D934C
:101FF0003C933AC02091770330917803232B41F42E
:102000002091FA023091FB023093780320937703FA
:102010002091F8023091F9022115310541F42DB7D4
:102020003EB74091FC025091FD02241B350BE0911C
:102030007703F0917803E217F307A0F42E1B3F0B10
:102040002817390778F0AC014E5F5F4F241735072A
:1020500048F04E0F5F1F50937803409377038193AE
:10206000919302C0E0E0F0E0CF01DF91CF910895BD
:102070000F931F93CF93DF93009709F48CC0FC015B
:102080003297138212820091790310917A0301151D
:10209000110581F420813181820F931F20917703F4
:1020A000309178032817390779F5F0937803E09396
:1020B000770371C0D80140E050E0AE17BF0750F47D
:1020C00012962D913C911397AD012115310509F11F
:1020D000D901F3CF9D01DA013383228360817181BD
:1020E000860F971F8217930769F4EC0128813981C5
:1020F000260F371F2E5F3F4F318320838A819B81BC
:1021000093838283452B29F4F0937A03E093790338
:1021100042C01396FC93EE931297ED0149915991A9
:102120009E01240F351FE217F30771F4808191811E
:10213000840F951F029611969C938E9382819381B2
:1021400013969C938E931297E0E0F0E0D8011296DC
:102150008D919C911397009719F0F8018C01F6CF9F
:102160008D919C9198012E5F3F4F820F931F20917C
:102170007703309178032817390769F4309729F4E9
:1021800010927A031092790302C013821282109384
:10219000780300937703DF91CF911F910F910895FA
:1021A000A0E0B0E0E6EDF0E10C946A0FEC010097DE
:1021B00021F4CB010E94A30FB8C0FC01E60FF71F6A
:1021C0009C0122503109E217F30708F4ACC0D90191
:1021D0000D911C91119706171707B0F005301105E6
:1021E00008F49FC0C80104978617970708F499C0A0
:1021F00002501109061B170B019311936D937C93E9
:10220000CF010E9438108DC05B01A01AB10A4C01A9
:10221000800E911EA0917903B0917A0340E050E0C6
:10222000E12CF12C109709F44AC0A815B905D1F595
:102230006D907C901197630182E0C80ED11CCA1486
:10224000DB0480F1A3014A195B096A0182E0C80E30
:10225000D11C1296BC9012971396AC91B5E0CB1698
:10226000D10440F0B282A38351834083D9016D939E
:102270007C930AC00E5F1F4FC301800F911FF901AD
:1022800091838083EB2DFA2FE114F10431F0D70113
:102290001396FC93EE93129744C0F0937A03E09365
:1022A00079033FC08D919C9111974817590708F405
:1022B000AC017D0112960D90BC91A02DB3CF809101
:1022C00077039091780388159905E1F4461757072D
:1022D000C8F48091F8029091F902009741F48DB70B
:1022E0009EB74091FC025091FD02841B950BE817AC
:1022F000F907C8F4F0937803E0937703F901718349
:1023000060830FC0CB010E94A30F7C01009759F09E
:10231000A801BE010E949F11CE010E943810C70182
:1023200004C0CE0102C080E090E0CDB7DEB7EEE0A1
:102330000C94860F81E090E0F8940C94AF11FB01AF
:10234000DC0102C001900D9241505040D8F7089531
:10235000FB01DC0101900D920020E1F7089513E0EC
:10236000C5EED3E004C0FE010E949D0F2196C63E3B
:08237000D107C9F7F894FFCF73
:102378000000000000000000000000000000000055
:102388000000000000000000000000000000000045
:10239800000000000000C0E0F0F8FCFCFEFFFCE0DC
:1023A8000000000000000000000000000000000025
:1023B8000000000000000000000000000000000015
:1023C8000000000000000000000000000000000005
:1023D8000000000000F8F8F8F8F8F8F8F8F8F8F84D
:1023E800F8F0F0E0E0C080C0FCFFFFFFFF7F3F7F18
:1023F800FFFFFFFFFF0000000000000000000000DA
:1024080000000000000000000000000000000000C4
:1024180000000000000000000000000000000000B4
:10242800000000000000000000000F1F3F7FFFFFBA
:10243800FFFFFFFFFFFFE7C7C7878F9F9FFFFFFFD4
:10244800C1C0E0FCFFFFFFFFFFFCFCFCFCFEFEFE42
:10245800FCFCF8F8F0E0C0C000000000000000003C
:102468000000000000000000000000000000000064
:102478000000000000000000000000000000000054
:102488000080C0E0F1FBFFFFFFFFFF7F1F0F0F87FA
:10249800E7FFFFFF1F1F3FF9F8F8F8F8F8F8FDFF0E
:1024A800FFFFFFFFFFFFFFFF7F3F0F070100000057
:1024B8000000000000000000000000000000000014
:1024C8000000000000000000000000000000000004
:1024D800000000F0FEFFFFFFFFFFFFFFFFFFFFFE12
:1024E8007E3F3F0F1FFFFFFFFCF0E0F1FFFFFFFF04
:1024F800FFFCF001010101010101010000000000E1
:1025080000000000000000000000000000000000C3
:1025180000000000000000000000000000000000B3
:10252800000000000000000303030303030303018A
:1025380001010100000000000000030F1F3F7F7F22
:10254800FFFFFFFF7F7F1F03000000000000000067
:102558000000000000000000000000000000000073
:10256800000000000000000000007B038000000065
:1025780000009B086C04EC056B04680B400B5C0BBB
:10258800500B6F0B6A0459065806FB0AB70A670A0C
:10259800490AD209730942545320534E202F20452B
:0A25A80043000D0A0031303030000E
:00000001FF
